:100000000F306500003066006400860190019101A8
:1000100092010130930094009501960198013B28CC
:10002000C830900003309100900B1428910B1428D5
:10003000640000346400051ADE288519DE280519DD
:10004000DE288518DE280518DE284034640085196E
:10005000DE280519DE288518DE280518DE2850342C
:1000600013188616131C861214180616141C061272
:1000700006138617803486018614861686150616A2
:100080000616861606178617102006128612061305
:100090008613063098001A201020980B4B2806145F
:1000A000861310201020102064000615FA309800E6
:1000B000861700008613000000000000000000000A
:1000C0000000000000000000000000000000980B8D
:1000D0005828FA30980086170000000000008613A8
:1000E0000000000000000000000000000000000010
:1000F00000000000980B6B28FA309800861700006B
:100100000000000000000000861300000000000056
:1001100000000000000000000000980B7E28FA306C
:10012000980086170000000000000000000000009A
:100130000000861300000000000000000000000026
:10014000980B9128FA3098008617000000000000F4
:100150000000000000000000000000008613000006
:10016000000000000000980BA428FA3098008617C1
:10017000000000000000000000000000000000007F
:10018000000000000000861300000000980BB72854
:10019000FA30980086170000000000000000000000
:1001A000000000000000000000000000000000004F
:1001B0008613980BCA2886171020DE28302064008A
:1001C0000518EF28851808290519212985193A29C4
:1001D000051A422915186F291218FA28DE28920AE2
:1001E0001020000000000518F12812180611121C3A
:1001F0005428DE2886130C3098001A201020980B03
:10020000FD28861710201A2010201A201020DE2822
:10021000930A10200000000085180A2913181329DA
:10022000131C1E29DE288616102086121020861622
:1002300010208612102086168615DE28861286115A
:10024000DE28940A10200000000005192329141844
:100250002C29141C3729DE2806161020061210201F
:10026000061610200612102006168614DE28061226
:100270008610DE2810200000000085193B29950A11
:100280001020DE28033098000613102026200617C1
:1002900010202620061310202620061710202620C6
:1002A0000613102026200617102026200613051EF0
:1002B000DE2812184229980B44290611051E6C29C4
:1002C00006168616061786171020061286120613C3
:1002D0008613102064005D2901309200DE281A2068
:1002E00006128612061386131A206430980006162A
:1002F00006120000000000000000980B77291A2069
:10030000643098000616000000000612000000008D
:10031000980B82291A20643098000616000000000D
:10032000000000000612980B8D291A2064309800F6
:1003300006160000000000000000980B98291A2003
:10034000643098008616861200000000000000004D
:10035000980BA2291A20643098008616000000002D
:10036000861200000000980BAD291A206430980016
:10037000861600000000000000008612980BB829C5
:100380001A2064309800861600000000000000006B
:10039000980BC3291A20643098000616000000004C
:1003A000000000000612980BCD291A206430980036
:1003B000061600000000061200000000980BD82965
:1003C0001A20643098000616061200000000000093
:1003D0000000980BE3291A206430980006170613D2
:1003E0000000000000000000980BEE291A20643085
:1003F0009800061700000000061300000000980B8C
:10040000F9291A2064309800061700000000000047
:1004100000000613980B042A1A206430980006176F
:100420000000000000000000980B0F2A1A20643022
:100430009800861600000000000000008612980B4D
:10044000192A1A20643098008616000000008612CF
:1004500000000000980B242A1A20643098008616A9
:1004600086120000000000000000980B2F2A1A20BE
:10047000643098008617861300000000000000001A
:10048000980B3A2A1A206430980086170000000062
:10049000861300000000980B452A1A20643098004B
:1004A000861700000000000000008613980B502AF9
:1004B0001A20643098008617000000000000000039
:1004C000980B5B2A1A206430980006170000000081
:1004D000000000000613980B652A1A20643098006B
:1004E000061700000000061300000000980B702A99
:1004F0001A20643098000617061300000000000060
:100500000000980B7B2A1A206430980086170000A0
:100510000000000000008613980B862A1A20643021
:100520009800861700000000861300000000980B5A
:10053000912A1A2064309800861786130000000064
:1005400000000000980B9C2A103098001A20102000
:10055000980BA62ADE28FF3FFF3FFF3FFF3FFF3FEC
:10056000FF3FFF3FFF3FFF3FFF3FFF3FFF3FFF3F9B
:10057000FF3FFF3FFF3FFF3FFF3FFF3FFF3FFF3F8B
:10058000FF3FFF3FFF3FFF3FFF3FFF3FFF3FFF3F7B
:10059000FF3FFF3FFF3FFF3FFF3FFF3FFF3FFF3F6B
:02400E00F73F7A
:08400000FF3FFF3FFF3FFF3FC0
:00000001FF
